:020000000143BA
:0100030032CA
:01000B0032C2
:0100130032BA
:01001B0032B2
:0100230032AA
:1800250075880075890075D00075A800227F000FEFB4FFFB227E000E6B
:18003D001132EE70FA2211257590FC113AE59023F590113AE59023F577
:1800550090113AE59023F590113AE59023F590113AE59023F590113A80
:18006D00E59023F590113AE59003F590113AE59003F590113AE590030B
:18008500F590113AE59003F590113AE59003F590113AE59003F59011F5
:03009D003A0145E0
:00000001FF
